:1000000070C0BAC188C087C086C085C084C083C0A4
:1000100082C081C080C07FC07EC07DC07CC07BC0EC
:100020007AC079C078C016032800530029004E001A
:10003000450053005F0075007300620018037200F2
:100040006100700068006E00650074002E006E0094
:100050006500740004030904090222000101008004
:100060003209040000010300000009210101000120
:100070002200000705810308000A120101010000A7
:1000800000088117960A0101010200010501090516
:10009000A1010901A10009300931150026FF0075F1
:1000A0000895028102C005091901290815002501DA
:1000B000750195088102C005010905A1010901A189
:1000C0000009300931150026FF00750895028102EC
:1000D000C005091901290415002501750195048140
:1000E00002C011241FBECFE5D4E0DEBFCDBF10E0BB
:1000F000A0E6B0E0E0E9FBE002C005900D92A43874
:10010000B107D9F710E0A4E8B0E001C01D92AB3C04
:10011000B107E1F753C374CFCF93DC01C62F693029
:1001200008F0C8E02BE490919C0090FD23EC8091B6
:10013000620087FF04C09F5F90939C0003C08FEF15
:10014000809362002093B500E6EBF0E02C2F215065
:100150002F3F19F08D918193FACF6C2F86EB90E0B1
:10016000BDD2CC5FC0936200CF9108951F93CF930F
:100170009091C500992309F483C0935097FD7EC0E8
:10018000E4E8F0E0E091B400EF5F40E0C0E8809187
:10019000C2008D3209F06EC0983009F06BC08081CA
:1001A000807609F064C021EB30E04093B10081819A
:1001B000882321F44093B20042E04EC0853021F400
:1001C00082818093C60048C0863091F5C0EC83815F
:1001D000813021F442E12AE730E03EC0823021F450
:1001E00042E228E530E038C0833099F482818823E8
:1001F00021F444E024E530E02FC0813021F448E1CF
:100200002CE330E029C0823039F546E126E230E0C7
:1002100023C0813221F449E02AE630E01DC0823259
:10022000D9F44091B3002091C9003091CA0014C0A4
:10023000883021F441E028EC30E00EC0893021F410
:1002400082818093C80008C08A3011F441E004C064
:100250008B3011F440939C003093C4002093C30072
:100260008781882339F48681841720F402C0CF0166
:1002700039D2482FC0939A00409364001092C50071
:10028000909164009F3F09F44FC08091630087FF05
:100290004BC0692F993008F068E0961B909364007A
:1002A0001BE480919A0080FD13EC8F5F80939A008D
:1002B000A9EAB0E0E091C300F091C400962F9150FC
:1002C00086FF13C09F3FB9F084919D012F5F3F4F80
:1002D000AF014F5F5F4F9150E157F04011F48091B3
:1002E000B3008C93D901FA01EDCF9F3F21F08191AA
:1002F0008D939150FACFF093C400E093C300772719
:10030000C62F693040F489EA90E0E8D19C2F9C5FC9
:10031000C83030F402C01EE192E08FEF8093640099
:100320001093A8009093630080B3857019F0109229
:100330009B0011C080919B00882369F494E680B3F0
:10034000857049F49150D9F781E080939B00909398
:10035000C6009093C100CF911F91089584E890E06A
:100360008093C0000B968093B40085B7836085BFEF
:100370008BB780648BBF08950F930FB70F93809B4B
:10038000FECF809B06C0809B04C0809B02C0000003
:1003900000C01F933F932F9331E014E000B3102768
:1003A00010FD32E0102F3A95C9F700FDE7C000B309
:1003B000102717952FE72795DF9310B3012707958F
:1003C0002795CF93C091C00000B3102717952795AC
:1003D0003BE0D0E04F9310B30127079527954FEFEF
:1003E000000055C0809BFECF809B06C0809B04C050
:1003F000809B02C0000000C0DF9100C0CDCF10B3D1
:10040000157079F1407C2C6F13C000B3057049F171
:1004100041782C6F15C0057021F1102F2C6F00B39F
:1004200019C000B30570E9F04E7F2C6F18C038F387
:1004300000B30570B1F0102717952795243028F3E5
:1004400010B3012707952795422749934FEF00B333
:10045000243008F3102717952795243010F310B394
:100460001570E1F10127079527952430F0F000B3CE
:100470000570A1F11027179527952430E0F010B3EF
:100480000127079527953A9541F12430D0F000B324
:10049000057021F11027179527952430C0F010B36F
:1004A0000127079527952430C2CF10B31570B1F0FE
:1004B0004C7F2C6FDCCF00B3057081F0487F2C6F30
:1004C000DECF10B3157051F0407F2C6FE0CF00B33A
:1004D000057021F0407E2C6FE2CF3DC03C2FC091D3
:1004E000C0003C1B00E433300ABFA8F10881198129
:1004F000412F1F772091C1000D3289F1013E79F122
:100500000936C1F00777033431F51091C700112384
:1005100011F10091C5000030D1F53430DAF130939B
:10052000C5001093C2000091B400C093B4000093C2
:10053000C00030C0121779F447FD3AC03091630013
:100540003F3F29F10FEF00936300C8EAD0E025C0D8
:1005500000270093C7004F91CF91DF910FC0121772
:10056000B9F70093C7000FEF009364000093630096
:100570004F91CF910AB706FD35CFDF9100E40ABF56
:100580002F913F911F910F910FBF0F911895C0E6CA
:10059000D0E002C0C1E6D0E032E05F9302B30A7F50
:1005A000016002BB55E011B3156011BB20E819C012
:1005B000309162003F3F59F30FEF00936200C5EBAB
:1005C000D0E0EBCF052710E002BB10C0052710E0FC
:1005D000089402BB13C0052710E015C0052710E0E2
:1005E00019C020FF052702BB279517951C3F50F720
:1005F00020FF0527279502BB17951C3F38F720FFE2
:1006000005272795179502BB1C3F28F720FF0527D4
:10061000279517951C3F02BB08F700C0499120FFA2
:10062000052702BB279517951C3F80F520FF05275E
:10063000279502BB17951C3F68F520FF05272795D6
:10064000179502BB1C3F58F520FF052727951795E6
:100650001C3F02BB38F5242F3A9519F60A7F5F91AB
:1006600002BB32E03A95F1F71091C600C256D04075
:1006700011F01093C100016011B31A7F02BB0A7F11
:100680004F91CF9111BB02BBDF9178CF052710E0CE
:1006900002BBCACF052710E0089402BBCDCF0527C7
:1006A00010E0CFCF052710E0D3CFA82FB92F8FEFC1
:1006B0009FEF41E050EA615070F02D9138E0722FC9
:1006C000782796958795269570FF02C084279527F1
:1006D0003A95A9F7F0CF809590950895E6DF8D9330
:1006E0009D930895FC012FE930E03093C4002093DE
:1006F000C3008081992780769070809719F5818159
:10070000813081F4E0919D00F0919E000484F58594
:10071000E02DC9010995E0919D00F0919E00808136
:1007200099270895823049F481EA90E09093C400BB
:100730008093C30081E090E008958A3019F48381AA
:100740008093A10080E090E00895EF92FF920F93D4
:100750001F93CF93DF93959AAC01415050408FEF98
:100760004F3F580721F180E3E82E85E7F82E012D51
:10077000112D959823E130E0C7010197F1F7215041
:10078000304037FFF9CF959AA0E3B5E7C0E0D0E05D
:1007900021E330E0CD010197F1F72150304037FFE0
:1007A000F9CF415050408FEF4F3F580711F7DF917D
:1007B000CF911F910F91FF90EF900895CFE5D4E076
:1007C000DEBFCDBFC0E001E01C2F8D9AB89A87B381
:1007D000897F87BB88B3866088BBC09880E395E734
:1007E0000197F1F786B3992786709070002E02C0AA
:1007F000959587950A94E2F78230910531F0039739
:1008000061F081E090E0A1DFFCCFA8D190939E0041
:1008100080939D0081E090E007C022D190939E00DC
:1008200080939D0082E090E090DFE0919D00F09148
:100830009E00848195819093CA008093C900828133
:100840008093B3009FEF95BB14BA8AEF82BB87E019
:1008500081BB80E08150F1F79150D9F782E081BBF4
:1008600085E083BF0680F781E02D099577DD7894D8
:10087000A8957CDC002349F0E0919D00F0919E005A
:100880000084F185E02D099500E008B600FE14C053
:1008900091E098BF8091A100882331F0153010F0CD
:1008A000155002C0182FC92FE0919D00F0919E00B5
:1008B0000084F185E02D0995E0919D00F0919E0066
:1008C0000284F385E02D0995882311F0C1E002C070
:1008D000CC2371F2809162008F3F51F6C0E0E0912D
:1008E0009D00F0919E000484F585E02D8FE990E055
:1008F0000995E0919D00F0919E0060818FE990E064
:100900000BDCB6CF90E0AC9A80E38A95F1F7AC9817
:1009100028E130E040E050E067E070E0822F8A9507
:10092000F1F7AD98990F9B9B9160822F8A95F1F713
:10093000AD9A6150704077FFF1CF9093A20028E10B
:1009400030E040E050E067E070E0822F8A95F1F7F8
:10095000AD9896959B9B9068822F8A95F1F7AD9AFA
:100960006150704077FFF1CF9093A3000895A49A4F
:10097000A59AA398AB9AAD9A95B3909585B3892320
:1009800085BBC0DF08958091730090917400892B1E
:1009900039F0109274001092730021E030E00BC027
:1009A00042E050E064EA70E082EA90E0E4D0282F70
:1009B000332727FD3095C9010895CF93DC01892B9A
:1009C00009F444C08091A200C091A30060E870E0E7
:1009D000FB01482F552740FF02C0EFEFF0E041FF39
:1009E00002C0E0E0F0E042FF02C06FEF70E043FFC2
:1009F00002C060E070E0EC93FD0161839A01220F78
:100A0000232F221F330B3195CA0180749070A5E00B
:100A100095958795AA95E1F7282BCA018072907069
:100A200073E0959587957A95E1F7282B4071507082
:100A300055954795242B8C2F99278F70907034E013
:100A4000880F991F3A95E1F7282B22838091A20005
:100A50009091A3009093A5008093A400CF91089556
:100A60008CE890E08638910509F0959890936A009B
:100A70008093690085E690E00895A49AA59AA398CA
:100A8000AB9AAD9A95B3909585B3892385BB0895AC
:100A900090E0AC9A80E38A95F1F7AC9828E130E0D9
:100AA00040E050E067E070E0822F8A95F1F7AD9862
:100AB000990F9B9B9160822F8A95F1F7AD9A6150B7
:100AC000704077FFF1CF9093A60008958091A60023
:100AD0009091A700891B992787FD90950895FC01A7
:100AE000892BB9F120E830E0B9018091A600482FA8
:100AF000552740FF02C06FEF70E041FF02C060E089
:100B000070E042FF02C02FEF30E043FF02C020E060
:100B100030E0608321839A01220F232F221F330BA1
:100B20003195CA018074907065E0959587956A95B6
:100B3000E1F7282BCA018072907033E09595879574
:100B40003A95E1F7282B4071507055954795242B25
:100B500022838091A6008093A700089587EB90E000
:100B60008638910509F0959890937A0080937900E2
:100B700085E790E00895FB01DC0104C08D910190B0
:100B8000801921F441505040C8F7881B990B0895F3
:100B90005AD2FFFFFF03002B000000B7048204C3FA
:100BA00004DD04010003002B0000003D054805663C
:040BB000056F0500C8
:00000001FF
